:1000000012C0189518951895189518951895189563
:100010001895189518951895189518951895189578
:100020001895189518958FE58DBFC0E2E8ED4E2E16
:1000300084E08EBFD4E0F3E05F2EEEEFF3E0A0E6C5
:10004000B0E088278D933197E9F787E189B980E09F
:1000500080BD88E18AB984B7082E877F84BF8FE18D
:1000600081BD87E081BD6624889889985FD041D2A0
:10007000ECE9FBE038D23DD2EAEEFBE034D239D2F3
:10008000EAE3FCE030D235D2EEE5FCE02CD231D20E
:10009000ECEAFCE028D22DD22CD24AD08FEF80930C
:1000A0006F008FEF809370008FEF809371008FEF60
:1000B0008093720082D0E1E0F0E022D280E0809371
:1000C0006F0080E08093700080E08093710080E09A
:1000D0008093720072D0E1E0F0E012D278D0002775
:1000E000A4E7B0E08C9187FB0EF401E041E0041737
:1000F00009F012C0E8EFFCE0F6D1FBD1E0E1FDE051
:10010000F2D1F7D198D007D1EDD08DE0F5D1E1E073
:10011000F0E0F6D1F7CF08C0E0E2FDE0E4D1E9D1AC
:10012000ECE3FDE0E0D1E5D1F894FFCFB3D408953E
:1001300021E780E091E0A0E6B0E00BD500916000FF
:10014000003009F0F5CF80E080936E0087E2809365
:100150006F0080E08093700080E08093710080E009
:100160008093720080E08093730086E08A9310E7AA
:10017000AEE6B0E0E5D48FE38093630086E0809341
:1001800064008BE5809365008FE48093660086E6CB
:10019000809367008DE6809368008DE78093690007
:1001A00087E080936A008FE780936B008FE68093EF
:1001B0006C0080E480936D00089581E080936E0070
:1001C00085E08A9310E7AEE6B0E0BAD4089567D42C
:1001D00018E97CD41CEA7AD412E078D46ED482E395
:1001E00090E09DD15CD418E971D41CEA6FD457D447
:1001F00019E96CD488D4A5E7B0E01C935ED4A5E7D8
:10020000B0E08C918F718C9300917500023009F0F1
:100210000CC08091740080688093740040D418E909
:1002200055D411E553D449D405C0809174008F771B
:1002300080937400089533D418E948D41AEA46D458
:100240002ED419E943D461D4A6E7B0E01C935BD463
:10025000A7E7B0E01C9331D4A6E7B0E08C91A8E703
:10026000B0E08D9388278C9391E0A8E7B0E045D269
:10027000A7E7B0E08C9187FBA8E7B0E08C9180F90C
:100280008C93A6E7B0E00C9107FB00270EF401E089
:1002900041E0041709F00CC0A8E7B0E00D911C91F3
:1002A00040E05EEF042B152BA8E7B0E00D931C9304
:1002B000E8E7F0E0D190E0808FEFE7FE8827F82EA6
:1002C000082F7ED2AAE7B0E0ACD2ECE8FBE053D333
:1002D000EAE7F0E051D2C5D2EDE0F0E0AAE7B0E005
:1002E000C3D30895A0ECB3E0AF93BF93EAE7F0E087
:1002F00043D224D111E001E0BF91AF9168D3E0EC8B
:10030000F3E0AEE7B0E0ABD3E0E7FDE0ECD0AEE782
:10031000B0E0E3D00895EAE7F0E02ED2E0E9FBE0B8
:100320002AD332D308F013C080916D0080936F0000
:10033000E4E9FBE020D3EAE7F0E01ED2E8D2EDE00A
:10034000F0E0E6D1A1E6B0E0DD92EC9225C0E8E96C
:10035000FBE011D3EAE7F0E00FD2D9D2EDE0F0E014
:10036000D7D1A1E6B0E0DD92EC920091610048EEB9
:1003700081D3A0E6B0E00C93A0E6B0E08C918F5F53
:100380008C93A0E6B0E0AD90BB24A2E6B0E0AA0D4D
:10039000BB1D8C9180936F00A1E6B0E00D911C9184
:1003A00048EE53E07ED0A1E6B0E00D931C9300919F
:1003B000610044E65FD3A0E6B0E00C93A0E6B0E0B5
:1003C0008C918F5F8C93A0E6B0E0AD90BB24A2E649
:1003D000B0E0AA0DBB1D8C9180937000A1E6B0E047
:1003E0000D911C9144E650E05CD0A1E6B0E00D9385
:1003F0001C93009161004AE03DD3A0E6B0E00C936D
:10040000A0E6B0E08C918F5F8C93A0E6B0E0AD9059
:10041000BB24A2E6B0E0AA0DBB1D8C9180937100B5
:10042000A1E7B0E08C9180688C93009161004AE074
:1004300021D3A0E6B0E08C93A0E6B0E08C918F5F72
:100440008C93A0E6B0E0AD90BB24A2E6B0E0AA0D8C
:10045000BB1D8C9180937200B0DE089500FC10D01B
:10046000089503D01ED001F8F9CF0024E89457FF77
:1004700002C009D0689400F80BD010F80124089548
:1004800002D009D00895509540954F5F5F4F089571
:10049000E89417FF0895009510950F5F1F4F68941B
:1004A0000895352F242FE894452B11F4689408956E
:1004B000512F402F0027112780E1440F551F001FA7
:1004C000111F021B130B416018F4020F131F4E7F04
:1004D0008A9599F70895A0ECB3E08D91882311F0E7
:1004E0000BD0FBCF089543D2802D11F005D0FBCF68
:1004F00008958DE001D08AE05D9BFECF8CB9089510
:1005000088EE93E00CD03197D9F708953197F1F741
:100510000895689462F80895E89462F80895EF9356
:10052000FF93EE27E82BE92B31F0E3E3F7E0319777
:10053000F1F70197D1F7FF91EF9108958DE207FD53
:100540008D938F2D881F802F881F8F57082F6894B9
:10055000F7F8802F87FF15C080958395082F80E3DB
:100560008D938EE28D93802F815228F080E38D93BE
:1005700099279C93089544270A95802F09F192D0DA
:100580001FC0805230F09EE49D9381E48D939D9333
:10059000EFCF4427DF92EF92FF920F938FE1801B02
:1005A00011F0082F7FD085D09EE29D930F91FF9090
:1005B000EF90DF9044270395003209F4D7CF27D07E
:1005C0003F93E4E4F6E038E12F2D1E2D0D2DFF249E
:1005D000EE24DD244427000F111F221F88F42F92E0
:1005E0003F92C5D1102CC3D1202CC1D1302CBFD10A
:1005F0003197410DD21CE31CF01C3F902F9001C09D
:10060000339631963A9539F73F9107D0B3CFDD0C49
:10061000EE1CFF1C0A95D9F70895002719E058D061
:100620008F93802B11F0039501C08F911A95B9F724
:10063000802F882309F49ACF8F91805D8D930A953E
:10064000D9F796CF0065CD1D80B2E60E40597307ED
:10065000A0ACB90350D6DC01286BEE0094357700CE
:10066000CA9A3B0065CD1D00B2E60E005973070023
:10067000ACB90300D6DC01006BEE0000357700005A
:100680009A3B0000CD1D0000E60E0000730700003D
:10069000B9030000DC010000EE000000770000005C
:1006A0003B000000F694E794D79447950A95D1F75C
:1006B000089500270DD08F9303958F2D8E298D29B6
:1006C000842BC1F78F91805D8D930A95D9F750CF18
:1006D0001F930F93002710E2440FDD1CEE1CFF1C3C
:1006E000001F802F9AE0890B10F0082F43951A9570
:1006F00099F7802F0F911F910895903041F00D913F
:100700001C91000F111F9A95E1F71C930E93089509
:1007100033D0992711278F2D880F80E8F82A802F52
:10072000881F08F41FEF41F08F57082F07FD04C002
:10073000003240F08FEF01C08827982FD82EE82E86
:10074000F82E09C08FE1801B082FF694E794D79408
:1007500097950A95D1F7112351F09095D094E09494
:10076000F09481E0980F8827D81EE81EF81E0F2D00
:10077000FE2CED2CD92E0895D190E190F1900191AD
:10078000089521913191419151910895102F90E850
:10079000FF0C001F0927990FF7941078652F90E838
:1007A000440F551F5927990F4795607800380895D1
:1007B000FF0C90E89027110F9795F794092F089553
:1007C000102FBD2CDE2CEF2CF02E11234AF4B09408
:1007D000D094E094F0949FEFB91AD90AE90AF90A83
:1007E0000EE1FF2039F4FE2CED2CDB2CBB2408504D
:1007F000C2F76BC032F00A95BB0CDD1CEE1CFF1C6F
:10080000F9CF01D0D5CFB7FE089590E8B91611F40D
:10081000D0FE08959FEFD91AE90AF90A09F4039561
:100820000895DD92ED92FD920C930895502F2D2D99
:100830003E2D4F2D612F08952DEC3CEC4CEC5DE3EB
:1008400066270FC099DFF2DFDD24EE2490E8F92E51
:100850000FE307C096DF05C02227332740E251E4AB
:100860006627552351F1002381F190DF71F116279E
:10087000005850580894050B18F407FD03C025C014
:1008800007FD23C0469537952795F694E794D794AE
:1008900022D0FF202AF0DD0CEE1CFF1C015073F06B
:1008A0009D2D969548F0DD203AF4EE202AF491E053
:1008B000D90E9927E91EF91E7BCF07C09FE7092FA4
:1008C000F92A9FEFD92EE92E0895DD24EE24FF2486
:1008D0000027112708959F929924AA24BB2488E118
:1008E000D216E306F40628F0D21AE30AF40A0894B2
:1008F00001C08894991CAA1CBB1CDD0CEE1CFF1CBB
:100900008A9571F7D92CEA2CFB2C9F9008953EDF35
:10091000E1F25038D1F21627005850580894051FBC
:1009200012F418F4CBCF08F0D0CF0AD0FF202AF071
:10093000BB0CDD1CEE1CFF1C3BCF0F5FFBF138CF67
:100940009F929924AA24BB24992788E1990CAA1C78
:10095000BB1CDD1CEE1CFF1C30F4920EA31EB41E4B
:10096000D91EE91EF91E8A9589F79F900895C895AA
:10097000319600200895FBDF202DF9DF302DF7DFC1
:10098000402DF5DF502D089507FB00680EF40F771A
:1009900057FB50680EF45F7707FD02C057FF05C094
:1009A000D216E306F406050708952D153E054F05FA
:1009B0005007089599278D9193958823E1F7939592
:1009C00011968C9311978E919A95D1F70895EA2FED
:1009D000FB2F00244C918D9103948E32E1F711246A
:1009E0008D9113948823E1F71A94101640F411970F
:1009F000202F2119239580E38D932A95E9F7113053
:100A000039F59927AE2FBF2FA00DB91FA00FB91F21
:100A10008C919C93853308F421C031E08E918E3205
:100A2000E9F38D3241F0830F8A3319F480E331E02A
:100A300001C033278C93AE1789F7332341F0AE2FD3
:100A4000BF2FB8DF81E34D3209F4319680830895DA
:100A50008827E00DF81FE00FF81F8083089581912B
:100A60008D938823E1F7089594E081918D939A9571
:100A7000E1F70895FF93881BF9E0001FFA9511F440
:100A8000FF910895881F841B18F4840F8894F5CF74
:100A90000894F3CFAC98AD98A498A5980895A59A1A
:100AA000A49803D0A59801D0A49AEF93FF93E5E012
:100AB000F0E02CDDFF91EF910895A59AA49AF5DF5F
:100AC000A5989D9BFECFF1DFA498EFCF0894111F4E
:100AD00001C0110F69F0A59A18F40000A49802C093
:100AE000A49A00C0E2DFA5989D9BFECFDEDFF1CF88
:100AF000A59AA498DADFA5989D9BFECFE8949C99CF
:100B0000689462F8D2CF089401C08894331F11E032
:100B1000A59AA498CADFA5989D9BFECFC6DF8894AE
:100B20009C990894111FA0F7A59A379510F4A498E2
:100B300001C0A49ABADFA5989D9BFECFB6DF0895A9
:100B4000AEDF1E7FC3DF89911D91C0DF8A95E1F77B
:100B5000B4CF122F803059F0A2DF1E7FB7DFAF93E2
:100B7000903059F0122F1160A9DF913011F4C3DFCA
:100B800001C0C3DF1D939A95C1F797CF00000040C5
:100B900000000000000020C1000020412020526120
:100BA0007070726573656E74617A696F6E652074BA
:100BB000656D70657261747572612073752064690A
:100BC00073706C61792037207365676D656E746929
:100BD0002C20636F6E20474D4D20414D3038202B27
:100BE00020474D4D2054535433004D6F6E74617245
:100BF00065204D696E69204D6F64756C6F2073754B
:100C0000205A322064656C6C6120474D4D2054534E
:100C100054332C20636F6C6C6567617265206C695E
:100C20006E6561204932432042555320616920633B
:100C30006F6D706F6E656E74690053414120313085
:100C40003634206520445320313633312C20636FF5
:100C50006D6520646120736368656D612E00496C69
:100C60002070726F6772616D6D61207072656C6566
:100C70007661206369636C6963616D656E7465207C
:100C80006C612074656D7065726174757261206449
:100C9000616C2073656E736F72652065206C6120D6
:100CA00072617070726573656E746100737569202E
:100CB000646973706C617920696E20666F726D6112
:100CC000206E756D65726963612C20636F6E206C98
:100CD00061207269736F6C757A696F6E65206469E3
:100CE00020302C352067726164692063656E7469F9
:100CF00067726164692E000053656E736F726520C0
:100D00004453313633312074726F7661746F2E0024
:100D100054656D7065726174757261202843290095
:100D200053656E736F726520445331363331206ED4
:100D30006F6E2074726F7661746F2100436F6E74F2
:100D4000726F6C6C61726520636F6C6C6567616D4E
:100D5000656E74692065207269657365677569726F
:100D60006520696C2070726F6772616D6D612E0015
:060D7000202020200000FD
:00000001FF
